:1000000001298200193400341534133411341234A8
:100010001C3400341A341834163414342734603441
:1000200000340034063402340034043451342134B2
:100030000034003400345A345334413457342234B9
:100040000034003443345834443445342434683460
:100050000034003420345634463454345234253479
:10006000003400344E3442344834473459345E341A
:100070000034003400344D344A34553426342A34A4
:10008000003400343C344B3449344F342934283460
:10009000003400343E343F344C343A3450345F340E
:1000A000003400340034403400345B343D340034D8
:1000B00000343B3403340D345D34003423340034D5
:1000C000003400345C3400340034003400342C3408
:1000D00000340034313400343434373400340034E4
:1000E000003430342E34323435343634383401343C
:1000F00067341B342B3433342D341E343934693493
:10010000003400340034003417341D34003400341B
:10011000003400340034003400340034003400343F
:10012000003400340734003400340A34003400341E
:10013000003400340034003400340034003400341F
:10014000053400340034003400340034003400340A
:1001500008340034003400340034003400340034F7
:1001600009340034003400340034003400340034E6
:1001700000340034003400340034003400340034DF
:1001800000340034003400340034003400340034CF
:100190000034003400342F34003400340034003490
:1001A00000340034003400340034003400340034AF
:1001B0000034003400346A34003400340034003435
:1001C000003400340034003400340034003400348F
:1001D000003400346134003465340E3400340034AB
:1001E00004340B3410346434003466346334003423
:1001F000003400340034623400341D340F341F34B2
:1002000000348316011481140115811581138611A0
:100210000612831206128615831686150616831299
:100220000612061E11298611831686118312861165
:1002300020306D22FF300022F6300022ED30002207
:10024000023098000022F4300022ED30002202300B
:1002500098000022ED300022023098000022F33096
:10026000002220300022F4300022F330002220301F
:1002700000228316061086100611831206148610BB
:1002800006154022FF302102031901290030210701
:1002900003194129FE30210203190129E13021020D
:1002A000031D7829402214302102031D42294022D7
:1002B00077302102031D42294022E1302102031D33
:1002C00042294022F0302102031D422940221430ED
:1002D0002102031D42294022F0302102031D422940
:1002E000402277302102031D42291F30DB214129A2
:1002F000A201E0302102031D97298030A200402294
:10030000F0302102031D8E294022123021020319F0
:10031000412959302102031DD129412912302102DE
:100320000319412959302102031D9D294129F0302B
:100330002102031D9D294022D129210A22070120E3
:10034000A200673022020319B2293B3022020319AE
:10035000B729693022020319BC292208003E031D77
:10036000DB2141291818AD2902309806C229181836
:10037000AD2904309806C22901309806181CC229FC
:100380006B30DD21ED300022180800229818CD29AD
:1003900006111819CF298610AD290615C92986140A
:1003A000CC29210A2207A2000120003E031941297D
:1003B000803EDB21412918180800910006102930E1
:1003C000920009309000920BE32929309200900BA3
:1003D000F92909309000061429309200920BEE2979
:1003E00029309200920BF22929309200920BF629C3
:1003F0000800910C031CFE290614E3290610E329CA
:100400009C001C08A1009A018615000006128316A4
:10041000861100000612831208309F00831686158D
:1004200083128619112A21180616211C0612A10C06
:1004300003189A0A861D1A2A9F0B112A86191E2A4A
:100440001A1806121A1C0616861D242A8619262A30
:100450000616861D292A83160616831286192E2A49
:10046000861D302A08306D2286118316861183126C
:1004700020306D224022FA302102031D012A08009B
:10048000A101861583168615831264008619452AF4
:10049000861D482A08309F0086194C2AA10C061A8E
:1004A000A117061EA113861D532A9F0B4C2A8619DD
:1004B000572A861D592A86195B2A861D5D2A8611B0
:1004C000831686118312861120306D2208009F004A
:1004D0006C229F0B682A0800FF30A000000000007B
:0A04E00000000000A00B6E2A0800C7
:00000001FF
